:1045CB0000000E0101180200000301FA0400FA05B5
:1045DB0000020A0A5A0B000F0C00FA0D00030E0022
:1045EB00030F0132100096120132130AFA14010262
:1045FB0015000217010A18010A1905321A010A1BC4
:10460B00010A1C053223011E2400642A00FA2B0028
:10461B00FA2C50782D003C2E00462F001E300064E3
:10462B003250783300003432FA3501643601643786
:10463B000150380A643C00643E003C3F000140FFDF
:10464B00FF411450420A5A430AC8440532450078C8
:10465B004600FA4701174802034C00FA4EFFFF5081
:10466B000404510596521432530B28540A965601E2
:10467B0002570546580002590A465A32FA5B010A9C
:10468B005C14325E000A5F00FE61FFFF64010B6782
:10469B0001036A0A3C6B00006C3296780132790197
:1046AB0032FAFAFA00000E0101180200000301FAB7
:1046BB000400FA0500020A0A5A0B000F0C00FA0D4F
:1046CB0000030E00030F0132100096120132130A81
:1046DB00FA14010215000017010A18010A19053214
:1046EB001A010A1B010A1C053223011E2400642A2D
:1046FB0000FA2B00FA2C50782D003C2E00462F0090
:10470B001E3000643250783300003432FA350164C5
:10471B00360164370150380A643C00643E003C3F6C
:10472B00000140FFFF411450420A5A430AC8440596
:10473B00324500784600FA4701174802024C00FA4E
:10474B004EFFFF500404510596521432530B28545C
:10475B000A96560101570546580001590A465A3226
:10476B00FA5B010A5C14325E000A5F00FE61FFFF18
:10477B0064010B6701036A0A3C6B00006C3296788C
:10478B000132790132FAFAFA0065006F0079008381
:10479B00008D009700A100AC00B600C000CA00D489
:1047AB0000DE00E800F2005B0063006A0072007A32
:1047BB00008200890091009900A100A800B000B808
:1047CB0000BF00C700CF00D600DF00E600EE00F60A
:1047DB0000400046004C00520059005F0065006B22
:1047EB0000710077007D00830089008F0095009C8D
:1047FB0000A200A800AE00B400BA00C000C600CCF6
:0C480B0000D200D900DF00E500EB00F156
:10009E00AE32AF33740F8E048F05FF1200858C3491
:1000AE008D35AE32AF33740F8E048F05FF124A9A20
:1000BE008C328D33E53345326013740FC39533FFA5
:1000CE00E49532FE8E328F337834124AE6E54FA82D
:1000DE0034B80015D395354010E54FC39535FFE480
:1000EE009534FE8E348F358010E54F2418C3953528
:1000FE00FFE49534FE8E348F35AE34AF3574186F01
:10010E004E700B753517753400754F018003754FA2
:10011E000022900079E0B40104C20B8002D20B9051
:10012E00007AE0B40104C20C8002D20C9000B7E059
:10013E0075F0DCA4FFAEF0740A8E048F05FF12007A
:10014E008590079FECF0A3EDF0A208401674038C87
:10015E00068D07124A7F7401124A7190079DEEF0C8
:10016E00A3EFF07E017F00900075E0124A7F9000B1
:10017E00B8E08E048F05FF120085740AFF12008509
:10018E008D389000C1E075F0DCA4FFAEF0740A8EDD
:10019E00048F05FF1200859007A3ECF0A3EDF090FD
:1001AE0000C3E060139000C3E0F5F0741684FF7E88
:1001BE0000EF9007ABF0800674649007ABF09000F0
:1001CE00A2E0B40B0874E3900064F080499000A2A2
:1001DE00E0B419129000B8E090477E124A62E493A0
:1001EE00900064F080309000A2E0B41E129000B82F
:1001FE00E090479C124A62E493900064F08017905E
:10020E0000A2E0B428109000B8E09047C6124A62EF
:10021E00E493900064F0900040E0C3940550227483
:10022E00019000BBF09000BDE0B402067401900096
:10023E00BDF09000ADE0D39402400674029000AD84
:10024E00F09000D5E0B40117900020740FF0A37465
:10025E00FFF0900022E4F0A3F074029000D5F0902D
:10026E0000D5E0B40341900022E0FEA3E0FF900031
:10027E0020E0FCA3E0FD124ADE7410124A7F7408DF
:10028E00124A71EF900061F0EF700674FF900061FA
:10029E00F074009000D5F0900021E0900062F09094
:1002AE000020E0900063F0900066E090002CF0904B
:1002BE00002CE0240C90002DF090002DE0D394182B
:1002CE00400B90002DE0C3941890002DF09000305C
:1002DE00E4F090002CE0B4180C9000307401F09013
:1002EE00002C7401F0900031E4F090002DE0B41871
:1002FE000C9000317401F090002D7401F0900066A6
:10030E00E0FE9000C9E02E900033F0900033E0D371
:10031E009418400B900033E0C39418900033F09083
:10032E000033E0B40C06740D900033F0900033E00F
:10033E00B418069000337401F0900033E0D3940C9F
:10034E00400D900033E0C3940C900034F0800A907E
:10035E000033E0240C900034F09000ACE090002EBE
:10036E00F090002EE0B40C06740D90002EF090006C
:10037E002EE0D3940C400D90002EE0C3940C900010
:10038E002FF0800A90002EE0240C90002FF022C255
:10039E0093C294C291C292C287C290E5B554EFF552
:1003AE00B5E5B554DFF5B5C296C295C2A0C297C2E7
:1003BE00A2C2A1E5B5547FF5B5E5B554BFF5B5E5D7
:1003CE00B554FBF5B5C20D7536469000AFE070051D
:1003DE00754802800375480390000874FFF0A374FB
:1003EE00DCF0900090E090000EF8E4F0E8A3F0C28C
:1003FE0012C21474C8900024F074C8900028F075CE
:10040E002500752400C208756B00E54AB409037512
:10041E004A00753B00900016E4F0A3F0754B1E7574
:10042E002700752600C210C21190079FE0FEA3E0C0
:10043E00FF7403124A7F7401124A7190079DEEF009
:10044E00A3EFF0C20390000CE4F0A3F0C21C22054F
:10045E003C2285A74E75A7109000ADE0B4031EA2F6
:10046E00D8B34002C293A2D9B34002C294A2DAB367
:10047E004002C291A2DBB34002C2928012A2D8B354
:10048E004004C293C291A2D9B34004C294C292A2B4
:10049E00DCB34002C287A2DDB34002C29075D840E1
:1004AE00854EA722900047E4936406600280FE7496
:1004BE00C89007A5F8E4F0E8A3F075B500758401BF
:1004CE0075A70075FF8075EF06900032E4F075C9D0
:1004DE001075A70F75A1C775A70075D90075CE0C3D
:1004EE0075A70F75F1FE75F2FF75F30775F4787544
:1004FE00A4BA75A5FF75A60775AE0075AFFF75D4C6
:10050E008175D5FF75D6FF75D7FF75A70075A2014A
:10051E0075A14775F80975D80075D90475A71075BA
:10052E00D80075D90475DA0975DB0975DC0975DD36
:10053E000975DE0975DF0975D84075A70075E608DF
:10054E0075E71075BC0175BE0475BD6C75BE07757B
:10055E00BDA075BE0875BD0175BC0075BB1875BC18
:10056E002075BA0875E88075D11375A70F75E1056A
:10057E0075E20075C740C293C294C291C292C287FF
:10058E00C290E5B554EFF5B5E5B554DFF5B5C296B5
:10059E00C295C2A0C297C2A2C2A1E5B5547FF5B55D
:1005AE00E5B554BFF5B5E5B554FBF5B575970075D2
:1005BE009780740A1200757597C0E59754207002E3
:1005CE0080F8758F0275A700D2AF75980075A90CCB
:1005DE0075A70F75AB4375ADFB75AC1E75A7107582
:1005EE00C91875CA0075CB0075C80475A700758942
:1005FE0012758E04758C00758A00C2A9D28C758D09
:10060E0000758B00D2ABD28E75D944753100753022
:10061E0000752D00752C00754500754600C2997544
:10062E0009C8750800122A2175B50074639007A5D4
:10063E00F8E4F0E8A3F0122CAD7509647508001209
:10064E002A21C21B90004FE0B40108A2B54002D28D
:10065E001B802E90004FE0B4021175A70F75F30F9B
:10066E0075A700A2A34002D21B801690004FE0B4E3
:10067E00030F75A70F75F31775A700A2A44002D23A
:10068E001BA21BB3500302077674089007A5F8E46B
:10069E00F0E8A3F0122B7C750964750800122A216C
:1006AE0074099007A5F8E4F0E8A3F0122B7C750905
:1006BE0064750800122A21740A9007A5F8E4F0E880
:1006CE00A3F0122B7C750964750800122A21740B95
:1006DE009007A5F8E4F0E8A3F0122B7C7509647579
:1006EE000800122A21740C9007A5F8E4F0E8A3F094
:1006FE00122B7C750964750800122A21740D90075F
:10070E00A5F8E4F0E8A3F0122B7C750964750800D7
:10071E00122A21740E9007A5F8E4F0E8A3F0122B2C
:10072E007C750964750800122A2174029000AEF0DF
:10073E0090004FE0900072F090004FE0B40108740A
:10074E000090007AF0801C90004FE0B40208740014
:10075E009000BDF0800D90004FE0B4030674009041
:10076E0000CAF0D21702084F9007A5E4F0A304F0D8
:10077E00122B7C750964750800122A2174029007E9
:10078E00A5F8E4F0E8A3F0122B7C75096475080057
:10079E00122A2174039007A5F8E4F0E8A3F0122BB7
:1007AE007C750964750800122A2174049007A5F857
:1007BE00E4F0E8A3F0122B7C750964750800122A88
:1007CE002174059007A5F8E4F0E8A3F0122B7C75D0
:1007DE000964750800122A2174069007A5F8E4F042
:1007EE00E8A3F0122B7C750964750800122A217497
:1007FE00079007A5F8E4F0E8A3F0122B7C750964C6
:10080E00750800122A2174019000AEF090004FE09E
:10081E00900072F090004FE0B40108740090007ADE
:10082E00F0801C90004FE0B4020874009000BDF000
:10083E00800D90004FE0B4030674009000CAF0C221
:10084E0017122E219000B8E07006740A9000B8F0CE
:10085E00900064E0700674E3900064F0120120E5ED
:10086E00B54401F5B5740690003EF0740190003F5A
:10087E00F07403900041F07404900042F0742290E2
:10088E000043F07405900044F0900040E0B404067C
:10089E007404900044F07403900045F074009000CE
:1008AE004AF0740090004BF0740190004CF074000C
:1008BE0090004DF074FF90004EF0743290013CF0B9
:1008CE00743490013DF0742D90013EF0743190011E
:1008DE003FF07420900140F07434900141F0744365
:1008EE00900142F07479900143F0746C900144F0E1
:1008FE007420900145F07420900146F07420900110
:10090E0047F07420900148F07420900149F0742053
:10091E0090014AF09000D4E0900061F090008BE0DE
:10092E00900062F090008CE0900063F0C212C2144E
:10093E0074C8900024F074C8900028F0C210C21140
:10094E00A2B6B39209A2B3B3920A7525007524001C
:10095E00753646754B1E90005DE4F07526197527A9
:10096E006490000874FFF0A374DCF0C20D754A00A9
:10097E00C20875290075280090000CE4F0A3F074ED
:10098E003A900765F074FD900766F0756C00900064
:10099E005EE4F0752B00752A00900010E4F0A3F0D1
:1009AE00900090E090000EF8E4F0E8A3F090007153
:1009BE00E075F032A4FFAEF090001EEEF0A3EFF063
:1009CE0090079FE0FEA3E0FF7403124A7F740112AA
:1009DE004A7190079DEEF0A3EFF075490174FA90FD
:1009EE00003AF0C21C756B00753B00C20EC20FC2FE
:1009FE001DC203754C00C204D205C206D207C2182E
:100A0E00C219D21A74FE900035F074FE900036F0C2
:100A1E00753700754300753900753D32753E0075AA
:100A2E003F00743C900038F0754000743C900039E3
:100A3E00F0754100754200900016E4F0A3F0754485
:100A4E0000D2B2D2A4D2B0D2B1D2A3D2A7D2A6D261
:100A5E00A5D2B7900071E0D394FA400674FA9000D4
:100A6E0071F07E017F00900063E0124A7F90006279
:100A7E00E02FFF50010E900020EEF0A3EFF0EFD329
:100A8E0094FFEE940F4007900020E4F0A3F0900046
:100A9E0061E0700674FF900061F09000AEE0D394B8
:100AAE0002400674019000AEF09000AFE070057544
:100ABE00480280037548039000B0E0D394014006CD
:100ACE0074009000B0F09000B6E0C3940A50067423
:100ADE000A9000B6F09000C0E0700674019000C05D
:100AEE00F09000C0E0B4FF0674FE9000C0F09000DD
:100AFE00C7E0D394FE400674FE9000C7F0740190D8
:100B0E0000CDF074019000CEF074009000D0F0741F
:100B1E00009000D5F0D29CD2EC75CF01A298B350C4
:100B2E0003020F17C298E54664046006E59964FF58
:100B3E006002801EE546600874E6254690003AF095
:100B4E00754600E545600874F0254590003AF0754D
:100B5E004500E5466003020C02754600E599B4FFB8
:100B6E0003754501E599B4FE03754502E599B4FD9B
:100B7E0003754503E599B4FC03754504E599B4FA8C
:100B8E0003754505E599B4FB03754601E599B4F97E
:100B9E0003754604E599D394E54007E599C394F0AF
:100BAE00400280168599477546027E017F00E54713
:100BBE00C394E6124A7F8E2E8F2F7531007530004A
:100BCE00E599D394C74007E599C394E64002801F88
:100BDE0085994775460374E5C39547F52F752E0025
:100BEE00AE2EAF2F9048171200647830124AC4D23E
:100BFE0099020F17E546B401028003020CDEE531BF
:100C0E004530700312039DAE30AF31900065124A2D
:100C1E00A6E599F07830124AE6AE30AF31EFB40166
:100C2E0006EEB407028003020CDE900765E0B43CCA
:100C3E00028003020CC8C29C120120900061E09059
:100C4E0000D4F0900062E090008BF0900063E09092
:100C5E00008CF0A2174031754F01E54FD394075029
:100C6E0025E54F9007A5F8E4F0E8A3F074AA9000EC
:100C7E0032F0122A4D750964750800122A21784F38
:100C8E00740126F650D4802F754F08E54FD3940E7D
:100C9E005025E54F9007A5F8E4F0E8A3F074AA906C
:100CAE000032F0122A4D750964750800122A217857
:100CBE004F740126F650D4122E2174C89007A5F851
:100CCE00E4F0E8A3F0D29C7546007545007599FBDB
:100CDE00E546B402028003020D72E531453070061E
:100CEE0085992D752C00AE30AF3174016F4E701B8F
:100CFE00AC2CAD2DAA2EAB2FED2BFBEC3AFA8A06BF
:100D0E008B07900065124AA6E599F07830124AE6F4
:100D1E00AE30AF3174026F4E704AAC2CAD2D740DE7
:100D2E006D4C702774639007A5F8E4F0E8A3F07497
:100D3E00AB900032F0900072E090004FF0122D86D2
:100D4E0074C89007A5F8E4F0E8A3F0AE2CAF2D74AC
:100D5E00566F4E700312039D1201208547997546FA
:100D6E0000754500E546B4033FAE30AF31900065E7
:100D7E00124AA6E599F07830124AE6AE30AF31ACA1
:100D8E002EAD2F8F028E038C068D079048531200C6
:100D9E0064E493F9740193FEEAD39EEB99400985BE
:100DAE004799754600754500E546B4040280030276
:100DBE000F17E5314530700312039DAE30AF319001
:100DCE000065124AA6E599F07830124AE6AE30AFC9
:100DDE0031EFB40006EEB401028003020F1790004B
:100DEE0048E075F002A4FDACF08D4FED9000651259
:100DFE004ABBEDFAE0FBEA900068124ABBEBFAE060
:100E0E00FBEA2BFA900048E0B502028003020F09BC
:100E1E000DED900065124ABBE54FFDE0FAED900036
:100E2E0069124ABBEAFDE0FAEDC39AFD900048E074
:100E3E00B505028003020F09E54F900067124ABB09
:100E4E00E54FFDE0FAED90006A124ABBEAFDE0FACA
:100E5E00ED2AFD900048E0B505028003020F09E57A
:100E6E004F90006B124ABBFDE0FAED900048E0F4A3
:100E7E00042A90004FF0E54F90006C124ABBFDE043
:100E8E00FAED900048E0F4042A900050F0E54F90FF
:100E9E00006D124ABBFDE0FAED900048E0F4042A22
:100EAE00900051F0E54F90006E124ABBFDE0FAED56
:100EBE00900048E0F4042A9007A5F8E4F0E8A3F0C7
:100ECE0074AB900032F0122D86750964750800120D
:100EDE002A219007A5124A8D122D86750964750870
:100EEE0000122A219007A5124A8D122D867599F9A6
:100EFE00750964750800122A2180FE7599FF75091F
:100F0E0064750800122A2180FEE5456006A299B399
:100F1E00B34003021095C299E545B4011FAE30AF40
:100F2E003190003E124AA6E0F5997830124AE6AEAC
:100F3E0030AF3174116F4E7003754500E545B40244
:100F4E0003854999E545B4031DAE30AF3190006578
:100F5E00124AA6E0F599EFB40107EEB40703754502
:100F6E00007830124AE6E545B404028003021057B9
:100F7E00E53145307003852599AE30AF3174016F80
:100F8E004E7003853799AE30AF3174026F4E7003D9
:100F9E00853999AE30AF3174036F4E7003853D992C
:100FAE00AE30AF3174046F4E7003853F99AE30AFE3
:100FBE003174056F4E7003854099AE30AF317406B3
:100FCE006F4E7003854199AE30AF3174076F4E701E
:100FDE0003854299AE30AF3174086F4E70069000A3
:100FEE0017E0F599AE30AF3174096F4E7006900070
:100FFE003AE0F599AE30AF31740A6F4E7003854307
:10100E0099AE30AF31740B6F4E7003853E99AE3092
:10101E00AF31740C6F4E7003854499AE30AF31749E
:10102E000D6F4E700590003AE4F0AE30AF31740D96
:10103E006F4E70037599FC7830124AE6AE30AF31C0
:10104E00740E6F4E7003754500E545B4053990007A
:10105E0040E0D394044010AE30AF319045CB124AED
:10106E00A6E493F599800EAE30AF319046AF124A9A
:10107E00A6E493F599AE30AF3174E36F4E700375FD
:10108E0045007830124AE6E54664016005E546B44F
:10109E000403020B27C28E7E107F00E53C124A7FAE
:1010AE00E58D75F010A4FDACF0EF2DFDEE3CFCE5EA
:1010BE008B75F01084FF7E00ED2FFFEC3EFE8E262A
:1010CE008F27D28E900092E06056900018124A8DB3
:1010DE00900018E0FCA3E0FD90001AE0FAA3E0FBFC
:1010EE00EDB5033CECB50238B216A208B34013A21C
:1010FE0016B34008E5B54404F5B58006E5B554FBD6
:10110E00F5B590001AE0FEA3E0FF90001CE0FCA3F2
:10111E00E0FDEF2DFDEE3CFC90001AECF0A3EDF09F
:10112E0090009FE0600990009FE0C394034002800E
:10113E006F124321A208B3500990005DE0C39428BA
:10114E0040028006900089E0F56AE56A75F005A414
:10115E00FFAEF09007A7EEF0A3EFF0900076E0C39D
:10116E0095394007E537C3953850079007A7E4F047
:10117E00A3F0AE57AF589007A7E0FCA3E0FDEFD366
:10118E009DEE9C4004C2A1800B90005DE0C3943C98
:10119E005002D2A190009FE0B40205A2A1B392A288
:1011AE0090009FE0B4031C12441DAE57AF58900739
:1011BE00A7E0FCA3E0FDEFD39DEE9C4004D2A180FE
:1011CE0002C2A190007AE06009A2B3300A01B3B363
:1011DE0040028039A2B3300A01B34031A2B3300CC1
:1011EE0001B3401C9000ADE0B40306A218B3B340A7
:1011FE00028006740590003AF0D218A20CB3920A3F
:10120E00A20CB330B301B34004A20C920AA2B630C2
:10121E000901B35003021775A2B6300901B350038A
:10122E00021775A2B6300B01B3500302168E754924
:10123E0000900092E07013A20BB34008E5B554FB8A
:10124E00F5B58006E5B54404F5B50536A20DB3B384
:10125E005013AE26AF27900008E0FCA3E0FDEDC3CF
:10126E009FEC9E4003021352E548B40330E536B4BA
:10127E001805754801801FA21CB3401AE536C394A9
:10128E0018500690003A7401F0E536D394184006D3
:10129E00740290003AF0753601D21C8044E548B4D1
:1012AE000206754801753618E536B418057536010F
:1012BE00802F90003AE0701AE536C39418500690CD
:1012CE00003A7401F0E536D394184006740290008B
:1012DE003AF09000AFE0B4020512039D800375361C
:1012EE0001AE28AF29AC26AD27EF2DFDEE3CFC74E8
:1012FE0003FF1200858C288D29900092E0604390A8
:10130E000018E0FEA3E0FF900092E08E048F05FF30
:10131E0012008574018C068D07124A7190001CEE26
:10132E00F0A3EFF090001CE0F8A3E090001AC8F0D4
:10133E00A3C8F0900018E4F0A3F0C216E5B554FB74
:10134E00F5B5802BAE28AF29AC26AD27EF2DFDEEDF
:10135E003CFC74018C068D07124A718E288F29ACC5
:10136E0026AD27EDD3944CEC941D400312039DE55E
:10137E0036B41810740390003AF09000AFE0B40247
:10138E000312039DAE2AAF2BAC26AD27EF2DFDEE3B
:10139E003CFC8C2A8D2BAE26AF27EFD39DEE9C40C6
:1013AE0011900010E0FAA3E0FBEBC394E8EA94037B
:1013BE0040028006900010124A8D90000CE0FEA3B1
:1013CE00E0FFAC26AD27EF2DFDEE3CFC90000CECC3
:1013DE00F0A3EDF09000AFE0B4021DAE26AF27747F
:1013EE0005124A7F74038E048F05FF12008590004C
:1013FE0008ECF0A3EDF08016AE26AF277403124A68
:10140E007F7401124A71900008EEF0A3EFF0C28EC5
:10141E00758D00758B00753C00752701752600D201
:10142E008EE536240575F00684AFF07E00EF4E7023
:10143E007590000CE0F8A3E090000AC8F0A3C8F085
:10144E0090000AE0FEA3E0FFEF4E600B7C7E7D2A4B
:10145E001249818E248F2590000CE4F0A3F0AE2467
:10146E00AF257428BE00039F5010E53B2FFF50019F
:10147E000E7401124A718E248F2585253B9000B67D
:10148E00E0A824B8000DD395254008E52590003737
:10149E00F080099000B6E014900037F0E548600641
:1014AE007525007524009000ADE0B4030890002E61
:1014BE00E0653660028026A218B34004D21980027D
:1014CE00B21990007AE0600BA218B35006A219B3BD
:1014DE00B340028006740490003AF0C218E53664F8
:1014EE00086005E536B4140990009FE060031240D1
:1014FE0063900033E065366007900034E0B5360344
:10150E00754A00A20E50030215F690006BE0B4016E
:10151E005AE53F75F00584FF7E00900565124AA6D8
:10152E00E0F533753200AE32AF33900069E0124A07
:10153E007F74648E048F05FF12008574C18C068D36
:10154E0007124A7F8E348F3590000EE0FEA3E0FF27
:10155E00AC32AD3312000374648E048F05FF12009B
:10156E008590000EECF0A3EDF0800F900069E07511
:10157E00F0C1A4FFAEF08E348F35E539C394CC5054
:10158E0006E53545347002805D75A71085F94F85E7
:10159E00FA507E017F00E550124A7FE54F2FFF5033
:1015AE00010E8E328F33AC34AD35EF2DFDEE3CFC9B
:1015BE008C348D35D293D294E535F5FBE534F5FCBC
:1015CE00E535F5E9E534F5EA9000ADE0B40314D263
:1015DE0091D292E535F5EBE534F5ECE535F5EDE533
:1015EE0034F5EE75A700D20EE548B40106E5366473
:1015FE00086002800F754B0190003D7401F0E5B557
:10160E004401F5B5E54870739000B2E0600D9000AE
:10161E00B9E0A824B800069525400280329000B2A9
:10162E00E0B4021790002CE06536600790002DE0C4
:10163E00B53603754B03754400800CC2007544002B
:10164E00900016E4F0A3F0740990003AF0802C900C
:10165E00002CE06536600790002DE0B53603754B23
:10166E000190002CE0B5360690003D7401F090001C
:10167E002DE0B53606740290003DF0A20BB3920930
:10168E00A20BB330B601B350030217757549019022
:10169E000092E07013A20BB34008E5B54404F5B513
:1016AE008006E5B554FBF5B5A20B9209E536D39449
:1016BE00494012D20DE536D394614009740390006F
:1016CE003AF07536469000BAE0B40107E542C3948D
:1016DE00144002800312039D742890005DF0A20452
:1016EE00300501B35017A204B34008E5B54408F520
:1016FE00B58006E5B554F7F5B5A2049205A20630FD
:10170E000701B35017A206B34008E5B54402F5B57C
:10171E008006E5B554FDF5B5A2069207E542C394E1
:10172E00415009740E90003AF012039D900044E06F
:10173E00FE900040E004C39E4009900040E0D39428
:10174E0006400974FB90003AF012039D900049E0A8
:10175E006015900049E0FE900043E06E600974FE53
:10176E0090003AF012039DA210B3B3500890002ED1
:10177E00E065366003021853A202B35006A200B30E
:10178E00B3400302184F75A71085F94F85FA507EA6
:10179E00017F00E550124A7FE54F2FFF50010E8E5C
:1017AE00328F33900014E0FCA3E0FDEF2DFDEE3CF4
:1017BE00FC8C348D359000ADE0B4034EA208B340DE
:1017CE0028A219B3400CE535F5FBE534F5FCD293B0
:1017DE00800AE535F5EBE534F5ECD291A203B34082
:1017EE0004D2A08002C2A0801FE535F5FBE534F5DA
:1017FE00FCE535F5EBE534F5ECD293D291A203B3CB
:10180E004004D2A08002C2A08011E535F5FBE5347C
:10181E00F5FCD293A203B34002D2919000CBE0B478
:10182E00021CAE32AF33AC55AD56EF2DFDEE3CFC87
:10183E008C348D35E535F5FDE534F5FED28775A78B
:10184E0000C210D211A211B3B3500890002FE06560
:10185E00366003021931A202B35006A200B3B340A0
:10186E000302192D75A71085F94F85FA507E017F59
:10187E0000E550124A7FE54F2FFF50010E8E328F3A
:10188E0033900014E0FCA3E0FDEF2DFDEE3CFC8C4C
:10189E00348D359000ADE0B4034EA208B34028A2BB
:1018AE0019B3400CE535F5E9E534F5EAD294800A32
:1018BE00E535F5EDE534F5EED292A203B34004D250
:1018CE00A08002C2A0801FE535F5E9E534F5EAE512
:1018DE0035F5EDE534F5EED294D292A203B3400481
:1018EE00D2A08002C2A08011E535F5E9E534F5EA13
:1018FE00D294A203B34002D2929000CBE0B4021C69
:10190E00AE32AF33AC55AD56EF2DFDEE3CFC8C3404
:10191E008D35E535F5CEE534F5CFD29075A700D2ED
:10192E0010C211E54BB40816123992A210B350052D
:10193E00A211B340028004D210D211754B1EE54B9A
:10194E00B4070612374A754B08E54BB4063D9000B6
:10195E000EE0FEA3E0FFEF4E6006A208B3B3400216
:10196E008023AE51AF5290000EE0FCA3E0FDEF2DB0
:10197E00FDEE3CFC8C518D52E536D3940C50069006
:10198E00000E12003912351C754B07E54BB40506D7
:10199E0012337C754B06E54BB404329000A0E090F8
:1019AE002A03F82828731230108012123010800D7E
:0D19BE001231BE80081232708003123270A8
:0F2A03000219B40219B90219BE0219C30219C887
:1019CB00900082E0600512414C8002C204754B0509
:1019DB00E54BB403028003021AC5900085E0600555
:1019EB0012423C8002C2069000A0E0D39402403F1A
:1019FB00900074E02403A824B800049525500990A6
:101A0B000076E0D3953950028008D202740890001A
:101A1B003AF0900074E0A824B80005D39525500B3C
:101A2B00900076E02403C395395002C202803990AE
:101A3B000074E02403A824B8000495255007E5376B
:101A4B00C3953840028008D202740890003AF09097
:101A5B000074E0A824B80005D395255009E5382477
:101A6B000FC395375002C2029000BAE07007E542EF
:101A7B00C3941440028002D202A2024005754B04AB
:101A8B00800A754B1E900016E4F0A3F0A208B34039
:101A9B0029E53F75F00584FF7E00900565124AA687
:101AAB00E0C394695005124098800F90079FE0F8AF
:101ABB00A3E090079DC8F0A3C8F0E54BB40A0280E1
:101ACB0003021B63900026E0C394465008C2967431
:101ADB0046900026F0900030E0B4011DE559240F2C
:101AEB00F5599007A1E0FEA3E0FF740F2FFF500103
:101AFB000E9007A1EEF0A3EFF085593375320090ED
:101B0B00002CE0F54F12009EE535900026F090007A
:101B1B0004E532F0A3E533F0E54F900027F0C21354
:101B2B009007A1E0F532A3E0F53390002CE0F54FE0
:101B3B0012009EE535900024F0900000E532F0A3F2
:101B4B00E533F0E54F900025F0C212E548B40105EE
:101B5B00754B0B8003754B03900024E0B53670A2D8
:101B6B0012404F900000E0FEA3E0FFEF4E6021AE6D
:101B7B0028AF29900000E0FCA3E0FD120003740FD6
:101B8B008E048F05FF120085900000ECF0A3EDF0A2
:101B9B00900025E0601A900000E0FEA3E0FFAC2867
:101BAB00AD29EF2DFDEE3CFC900000ECF0A3EDF029
:101BBB00D212AE26AF27900000E0FCA3E0FDEFC3EE
:101BCB009DEE9C400AD296C21274C8900024F0A2DB
:101BDB0012B3B35007900024E0B53602800AD296B8
:101BEB0074C8900024F0C212900026E0B53670A2A3
:101BFB0013404F900004E0FEA3E0FFEF4E6021AED8
:101C0B0028AF29900004E0FCA3E0FD120003740F41
:101C1B008E048F05FF120085900004ECF0A3EDF00D
:101C2B00900027E0601A900004E0FEA3E0FFAC28D0
:101C3B00AD29EF2DFDEE3CFC900004ECF0A3EDF094
:101C4B00D213AE26AF27900004E0FCA3E0FDEFC358
:101C5B009DEE9C400AC2967446900026F0C213A2D9
:101C6B0013B3B35007900026E0B53602800AC29634
:101C7B007446900026F0C213E54BB40B02800302AE
:101C8B001D3690002AE0C3944650139000BBE0B47D
:101C9B000104C2968002C295744690002AF090000F
:101CAB0031E0B4011DE559240FF5599007A1E0FE71
:101CBB00A3E0FF740F2FFF50010E9007A1EEF0A3CE
:101CCB00EFF085593375320090002DE0F54F12007F
:101CDB009EE53590002AF0900006E532F0A3E5333F
:101CEB00F0E54F90002BF0C2159007A1E0F532A361
:101CFB00E0F53390002DE0F54F12009EE535900096
:101D0B0028F0900002E532F0A3E533F0E54F9000A8
:101D1B0029F0C214E548B4010F75480074C890004F
:101D2B0024F074C8900028F0754B03900028E0B5A0
:101D3B00367BA214404F900002E0FEA3E0FFEF4E73
:101D4B006021AE28AF29900002E0FCA3E0FD120059
:101D5B0003740F8E048F05FF120085900002ECF0C8
:101D6B00A3EDF0900029E0601A900002E0FEA3E0E2
:101D7B00FFAC28AD29EF2DFDEE3CFC900002ECF002
:101D8B00A3EDF0D214AE26AF27900002E0FCA3E047
:101D9B00FDEFC39DEE9C40159000BBE0B40104D257
:101DAB00968002D295C21474C8900028F0A214B386
:101DBB00B35007900028E0B5360280159000BBE0C9
:101DCB00B40104D2968002D29574C8900028F0C258
:101DDB001490002AE0B5367BA215404F900006E028
:101DEB00FEA3E0FFEF4E6021AE28AF29900006E086
:101DFB00FCA3E0FD120003740F8E048F05FF12008D
:101E0B0085900006ECF0A3EDF090002BE0601A90AB
:101E1B000006E0FEA3E0FFAC28AD29EF2DFDEE3C64
:101E2B00FC900006ECF0A3EDF0D215AE26AF279098
:101E3B000006E0FCA3E0FDEFC39DEE9C4015900077
:101E4B00BBE0B40104C2968002C295744690002A8E
:101E5B00F0C215A215B3B3500790002AE0B53602B5
:101E6B0080159000BBE0B40104C2968002C2957449
:101E7B004690002AF0C215E54BB402028003021F04
:101E8B0028123DFB123F1290079DE0FEA3E0FF746A
:101E9B000A124A7F90000AE0FCA3E0FD74098F024E
:101EAB00FF1200858D078C038E048A058B06124961
:101EBB00819007A1EEF0A3EFF09000BBE0B4010816
:101ECB007478BE00059F4002800D74789007A1F8CE
:101EDB00E4F0E8A3F0801B9007A1E0FEA3E0FF7401
:101EEB00F0BE00039F500B74F09007A1F8E4F0E8EC
:101EFB00A3F09007A1E0FEA3E0FFE5592FFF5001EF
:101F0B000E9007A1EEF0A3EFF090003DE0B40103BB
:101F1B00754B0A90003DE0B40203754B0BE54BB4D7
:101F2B0001259000D2E0902A12F8282873123B99D1
:101F3B008012123B99800D123C238008123CCF80FB
:041F4B0003123CCF72
:0F2A1200021F38021F3D021F42021F47021F4CC6
:101F4F00754B029000BDE0B40202800302206A903C
:101F5F000060E0D3953E5064900060E0F404253EAD
:101F6F00FE9000C0E08E00F5F0E884FF7E008F4FFA
:101F7F00EFC39410500CEF854FF0A4FDACF08D4FD4
:101F8F008003754FFF900060E0D3954F400B90009A
:101F9F0060E0C3954FF54C8003754C009000DBE07B
:101FAF00D3954C40069000DBE0F54C9000DCE0C38D
:101FBF00954C50069000DCE0F54C8071900060E08D
:101FCF00C3953EFE9000C0E08E00F5F0E884FF7EE2
:101FDF00008F4FEFC39410500CEF854FF0A4FDAC62
:101FEF00F08D4F8003754FFF854F33753200900092
:101FFF0060E02533FFAE3250010E8E328F3374FF07
:10200F00BE0009D39F400585334C8003754CFF906C
:10201F0000DBE0D3954C40069000DBE0F54C9000E0
:10202F00DCE0C3954C50069000DCE0F54CA208B301
:10203F00B350099000C8E0D3954D5002800A740741
:10204F0090003AF0C297801375A710E5CDC3954C59
:10205F004004C2978002D29775A700E54AC394093E
:10206F0040030227A5A2EDB350030227A5C2EDE559
:10207F004A600302221990006EE07003022208905A
:10208F0000A4E0B401028003022168900033E0B5A0
:10209F00360280030221657E017F00E5BE124A7F72
:1020AF00E5BD2FFF50010E8E328F3390006EE0B4DE
:1020BF0001187410124A7F900064E08E048F05FFA0
:1020CF00120085ED900035F0802CAE32AF337410D6
:1020DF00124A7F900064E08E048F05FF12008590F6
:1020EF000035E02DFD50010C74018C068D07124A4E
:1020FF0071EF900035F0E54360089000CAE064028C
:10210F00600280219000CCE0B4011A900035E07598
:10211F00F0E7A4FFAEF0E5438E048F05FF120085B4
:10212F00ED900035F0900035E0FE900036E0D39E44
:10213F004004D21A8002B21A900035E0900036F0B7
:10214F009000A0E064016006A21AB3B340028006BB
:10215F00900035E0F537022206D21A7E017F00E5A6
:10216F00BE124A7FE5BD2FFF50010E8E328F339086
:10217F00006EE0B401187410124A7F900064E08E74
:10218F00048F05FF120085ED900035F0802CAE32E4
:10219F00AF337410124A7F900064E08E048F05FFF6
:1021AF00120085900035E02DFD50010C74018C0656
:1021BF008D07124A71EF900035F0E54360089000EB
:1021CF00CAE06402600280219000CCE0B4011A9052
:1021DF000035E075F0E7A4FFAEF0E5438E048F0500
:1021EF00FF120085ED900035F09000A0E0640160D3
:1021FF0006900035E0F537800375370090006AE0F0
:10220F007005754A01800375BB18E54AB401028059
:10221F00030223BB90006AE070030223AA7E017FB2
:10222F0000E5BE124A7FE5BD2FFF50010E8E328FA3
:10223F00339000B0E0B4010F7E0F7FFFAC32AD33AF
:10224F00124ADE8E328F339000D5E0B40245AE32A3
:10225F00AF33900020E0FCA3E0FDEDD39FEC9E4058
:10226F000A900020E532F0A3E533F0AE32AF3390A1
:10227F000022E0FCA3E0FDEFD39DEE9C400A90000E
:10228F0022E532F0A3E533F0AE32AF337404124AD5
:10229F00718F399000D5E0704CAE32AF3390002083
:1022AF00E0FCA3E0FDEFD39DEE9C4009124ADE8EC9
:1022BF00328F338006753300753200AE32AF337410
:1022CF0010124A7F900061E08E048F05FF12008587
:1022DF008C328D337400D39D74019C400585333946
:1022EF0080037539FF9000A0E0B401028003022340
:1022FF00A8A208B3B3500E900074E0A824B800054C
:10230F00D39525500302239D900075E075F019A415
:10231F00FFAEF09000B8E08E048F05FF120085909D
:10232F0000B1E08539F0A4FFAEF074648D028C0328
:10233F008E048F05FF120085EA2DFDEB3CFC8C32DD
:10234F008D33E543600F9000CAE0B402089000CCD3
:10235F00E0640160028017AE32AF3374E7124A7F38
:10236F00E5438E048F05FF1200858C328D3390006C
:10237F0035E0A832B8000AD395334005853337804E
:10238F000BA21AB34006900035E0F537800BA21A66
:10239F00B34006900035E0F53780037539009000A3
:1023AF006DE07005754A02800375BB19E54AB402EA
:1023BF0002800302247690006DE07003022465E52D
:1023CF0036D3940C400302246390001EE0FEA3E07A
:1023DF00FFE53D124AD690001EEEF0A3EFF07E010E
:1023EF007F00E5BE124A7FE5BD2FFF50010E8E32F2
:1023FF008F339000DAE07013740A124A7F74518E93
:10240F00048F05FF1200858D3D8019AE32AF3374F6
:10241F000A124A7F8F048E057E017F95CDCCCD1297
:10242F0049818F3DE53DD394644003753D64900031
:10243F001EE0FEA3E0FFE53D2FFF50010E90001EB2
:10244F00EEF0A3EFF0900071E0048E048F05FF1201
:10245F0000858D3D8003753D329000BDE0700575A0
:10246F004A03800375BB13E54AB4035E9000BDE0D9
:10247F0060477E017F00E5BE124A7FE5BD2FFF500A
:10248F00010E8E328F337404124A718F3E9000BF4B
:10249F00E0853EF0A4FDACF07464FF1200858D3E24
:1024AF009000BEE0853EF0A4FFAEF074FF8E048F67
:1024BF0005FF1200858D4D8003753E0090006BE087
:1024CF007005754A04800375BB17E54AB404028092
:1024DF000302257790006BE0B4017C7E017F00E55D
:1024EF00BE124A7FE5BD2FFF50010E7404124A71D0
:1024FF008E328F33900038E06012900038E01490E5
:10250F00488F93A832B8000695334002800690009A
:10251F0038E014F0900038E0C394775013900038EF
:10252F00E00490488F93A832B80005D3953350023A
:10253F008006900038E004F0900038E0FE900091A3
:10254F00E08E0088F0A4FFAEF074648E048F05FF58
:10255F001200858D3F8003753F0090006CE0700581
:10256F00754A05800375BB16E54AB4050280030260
:10257F00260A90006CE0B4017C7E017F00E5BE125C
:10258F004A7FE5BD2FFF50010E7404124A718E323F
:10259F008F33900039E06012900039E014904908B1
:1025AF0093A832B80006953340028006900039E0B8
:1025BF0014F0900039E0C394775013900039E00481
:1025CF0090490893A832B80005D39533500280067E
:1025DF00900039E004F0900039E0FE900097E08E13
:1025EF000088F0A4FFAEF074648E048F05FF120014
:1025FF00858D40800375400075BB1FE54AB40633D7
:10260F007E017F00E5BE124A7FE5BD2FFF50010E10
:10261F008E328F337409124A7F74E68E048F05FF52
:10262F001200858D42900073E07005754A07800394
:10263F0075BB15E54AB40702800302274C9000735F
:10264F00E0700302273B7E017F00E5BE124A7FE563
:10265F00BD2FFF50010E8E328F337404124A718FCB
:10266F0041900073E0B401159000C7E08541F0A4DC
:10267F00FFAEF07407124A71EF9007AAF090007343
:10268F00E0B402159000C7E08541F0A4FFAEF074EE
:10269F0007124A71EF9007A9F0900073E0B403029C
:1026AF0080030227399000B4E0701CE541C3940AFF
:1026BF005002D201E541D394644002C201900093CD
:1026CF00E090005FF08063900093E070349000C75B
:1026DF00E08541F0A4FFAEF074FF8E048F05FF126A
:1026EF000085ED90005FF0AE24AF25741EBE00068E
:1026FF00D39F4002D201E539D394E54002C2018055
:10270F0029E541C3940A500DAE24AF25741EBE00B7
:10271F0004D39F50028002D201E539D394E54002E1
:10272F00C201900093E090005FF08003754100902C
:10273F0000CAE07005754A08800375BB14E54AB4FA
:10274F0008509000CAE060397E017F00E5BE124A52
:10275F007FE5BD2FFF50010E8E328F33EFD39421C3
:10276F00EE940E40057543FF8015AE32AF337410F3
:10277F00124A7F74E38E048F05FF1200858D43800C
:10278F000375430090006EE0600575BB1A800375FA
:10279F00BB18054AD2ECAE26AF27EFD39498EE9430
:1027AF003A5003022A00C20D7536469000AFE07012
:1027BF00057548028003754803C293C294C291C243
:1027CF0092C287C290E5B554EFF5B5E5B554DFF584
:1027DF00B5C296C295C2A0C297C2A2C2A1E5B55416
:1027EF007FF5B5E5B554BFF5B5A21BB34008E5B508
:1027FF004404F5B58006E5B554FBF5B5A20FB3500B
:10280F000EE539D394334007E539C394CC40030226
:10281F0028AAE5B54401F5B5742890005DF0900045
:10282F0069E075F064A4FFAEF08E348F357402BE8C
:10283F00000AD39F400675350275340075A71085C1
:10284F00F94F85FA507E017F00E550124A7FE54F20
:10285F002FFF50010E8E328F33AC34AD35EF2DFD7F
:10286F00EE3CFC8C348D35D293D294E535F5FBE5F7
:10287F0034F5FCE535F5E9E534F5EA9000ADE0B463
:10288F000314D291D292E535F5EBE534F5ECE5354D
:10289F00F5EDE534F5EE75A700D20FE539C3941ABF
:1028AF005002C20F90000874FFF0A374DCF0900088
:1028BF0090E090000EF8E4F0E8A3F0C212C2147496
:1028CF00C8900024F074C8900028F0C210C211758F
:1028DF002500752400753B00C208756B009000162B
:1028EF00E4F0A3F0754B1E90079FE0FEA3E0FF748A
:1028FF0003124A7F7401124A7190079DEEF0A3EF05
:10290F00F0900082E0600512414C8002C2049000FA
:10291F0085E0600512423C8002C206A20430050128
:10292F00B35017A204B34008E5B54408F5B58006C7
:10293F00E5B554F7F5B5A2049205A206300701B329
:10294F005017A206B34008E5B54402F5B58006E579
:10295F00B554FDF5B5A2069207C203752B00752A73
:10296F0000900010E4F0A3F0900071E075F032A435
:10297F00FFAEF090001EEEF0A3EFF090000CE4F02D
:10298F00A3F0C21C90005EE0C3943C5019758DA556
:10299F00758B00753C03E54AB4090990005EE004AD
:1029AF00F0754A00803BE54AB40903754A00752764
:1029BF0000752600758D00758B00753C0090005DCD
:1029CF00E0C3943C500890005DE004F08006743C36
:1029DF0090005DF090005DE0B43C06E5B554FEF567
:1029EF00B5E542C394415009740E90003AF01203BA
:0429FF009D020B2703
:104817000000010001400160018001A001C001E02A
:1048270002000300039603B603D603F40400050051
:1048370005180530054805600578059005A805C0E9
:10484700060006140628063C066E068C00FF013F8C
:10485700015F017F019F01BF01DF01FF02FF039598
:1048670003B503D503F303FF04FF0517052F05471A
:10487700055F0577058F05A705BF05FF0613062703
:10488700063B066F068B06A9DAD8D7D5D4D2D0CF88
:10489700CDCBC9C7C6C4C2C0BEBCBAB8B5B3B1AF29
:1048A700ADABA8A6A4A2A09D9B99969492908D8B40
:1048B70089878482807E7C79777573716F6D6B6968
:1048C700676563615F5D5B5957565452504F4D4B57
:1048D7004A4847454442413F3E3C3B3A39373635E3
:1048E700343231302F2E2D2C2B2A29282726252507
:1048F7002423222121201F1E1E1D1C1C1B1A1A19CE
:1049070019EEECEBEAE9E8E7E5E4E3E1E0DEDDDB1D
:10491700D9D8D6D4D2D0CECCCAC8C6C3C1BFBCBAE8
:10492700B7B5B2B0ADABA8A5A3A09D9B9895929043
:104937008D8A8785827F7D7A7775726F6D6A6865E4
:1049470063615E5C5A575553514F4D4B4947454339
:1049570042403E3C3B393836353332312F2E2D2BF2
:104967002A292827262524232221201F1E1D1D1C16
:0A4977001B1A1A1918181716161546
:102A2100750B00750A00AE0AAF0BAC08AD09EDC31A
:102A31009FEC9E401674FF12007575CF01780B74E0
:102A41000126F6500418E436F650DB22900032E0FD
:102A5100B4AA1C900765E0B43C159007A5E0FEA35D
:102A6100E0FFEF4E6009741EBE0004D39F500302C5
:102A71002B7B75350075340075F8099007A5E0FECC
:102A8100A3E0FF74076F4E6006740E6F4E700674FC
:102A91003A900765F09007A5E0FEA3E0FF7408BE39
:102AA100001ED39F401A7E017F089007A5E0FCA37A
:102AB100E0FD1DBDFF011C1200038E328F33801F0C
:102AC1009007A5E0FEA3E0FF7408124AD68F048E9A
:102AD100057E017F08CDCCCD1200038E328F33AE3F
:102AE10034AF35740CD39F74019E5003022B76A230
:102AF100F9B3407EE5354534700375A382AE34AF3A
:102B01003574016F4E700375A300AE34AF35740296
:102B11006F4E700D9007A6E075F002A4FDACF08D2C
:102B2100A3AE34AF3574036F4E700375A300AE349A
:102B3100AF357403BE00039F5013AC32AD33ED2F9C
:102B4100FFEC3EFE900061124AA6E0F5A3AE34AF61
:102B510035EFB40B09EEB401057414120075AE34EF
:102B6100AF35EFB40B07EEB4010375F80D783412ED
:102B71004AE6022AE0900032E4F02275350075340D
:102B81000075F8099007A5E0FEA3E0FF7408BE00F8
:102B91001ED39F401A7E017F089007A5E0FCA3E0A9
:102BA100FD1DBDFF011C1200038E328F33801F906B
:102BB10007A5E0FEA3E0FF7408124AD68F048E0534
:102BC1007E017F08CDCCCD1200038E328F33AE341F
:102BD100AF357411D39F74019E5003022CACA2F93E
:102BE100B35003022CA9E5354534700375A3D2AE69
:102BF10034AF3574016F4E700375A300AE34AF3539
:102C010074026F4E700D9007A6E075F002A4FDAC42
:102C1100F08DA3AE34AF3574036F4E700375A3000E
:102C2100AE34AF3574046F4E700375A300AE34AF8C
:102C31003574056F4E700375A300AE34AF3574065D
:102C41006F4E700375A300AE34AF3574076F4E70CD
:102C51000375A300AE34AF3574086F4E700375A3CE
:102C610000AE34AF357408BE00039F5016AC32ADD0
:102C710033ED2FFFEC3EFE90005C124AA6E5A3F077
:102C810075A300AE34AF35EFB41009EEB40105748D
:102C910014120075AE34AF35EFB41007EEB4010372
:102CA10075F80D7834124AE6022BCF22753500757E
:102CB100340075F809AE34AF357417BE0004D39FE4
:102CC1005003022D85A2F9B35003022D82E535454B
:102CD10034700375A3D2AE34AF3574016F4E7003F7
:102CE10075A300AE34AF3574026F4E700D9007A618
:102CF100E075F002A4FDACF08DA3AE34AF357403E2
:102D01006F4E700375A300AE34AF3574046F4E700F
:102D11000375A300AE34AF3574056F4E700375A310
:102D210000AE34AF3574066F4E700375A300AE3438
:102D3100AF3574076F4E700375A300AE34AF3574B1
:102D4100086F4E700375A300AE34AF357408BE0032
:102D5100039F500C900046124AA6E5A3F075A3000C
:102D6100AE34AF3574166F4E70057414120075AE23
:102D710034AF3574166F4E700375F80D7834124AFE
:102D8100E6022CB622900032E0B4AB028003022EA0
:102D91002075350075340075F809AE34AF357412FD
:102DA100BE007CD39F4078A2F9B34070E53545342D
:102DB100700375A382AE34AF3574016F4E70037525
:102DC100A300AE34AF3574026F4E700D9007A6E0CC
:102DD10075F002A4FDACF08DA3AE34AF3574036F72
:102DE1004E700375A300AE34AF357403BE00039F6C
:102DF100500990004B124AA6E0F5A3AE34AF3574EA
:102E0100116F4E70057414120075AE34AF35741124
:102E11006F4E700375F80D7834124AE6022D9B222D
:102E210090003BE4F074649007A5F8E4F0E8A3F0A7
:102E3100122CAD74C89007A5F8E4F0E8A3F0900057
:102E410052E0B4371A90004FE0900046F0900050E5
:102E5100E0900047F0900051E0900048F0804690EB
:102E6100003B7401F074659007A5F8E4F0E8A3F065
:102E7100122CAD74C89007A5F8E4F0E8A3F0900017
:102E810052E0B4371A90004FE0900046F0900050A5
:102E9100E0900047F0900051E0900048F080067407
:102EA1000290003BF090003CE4F074669007A5F8B6
:102EB100E4F0E8A3F0122CAD74C89007A5F8E4F093
:102EC100E8A3F0900051E0B4371290004FE0900079
:102ED10040F0900050E0900049F0807690003C7402
:102EE10001F074679007A5F8E4F0E8A3F0122CADA7
:102EF10074C89007A5F8E4F0E8A3F0900051E0B49D
:102F0100371290004FE0900040F0900050E09000A8
:102F110049F0803E740290003CF074689007A5F877
:102F2100E4F0E8A3F0122CAD74C89007A5F8E4F022
:102F3100E8A3F0900051E0B4371290004FE0900008
:102F410040F0900050E0900049F08006740390003A
:102F51003CF022E55C2533FFAE3250010E90006556
:102F6100124AA6E0F55DE55C2533FFAE3250010E55
:102F71000FBF00010E900065124AA6E0F55E856460
:102F810060E55DB55E05855D5C8041E55ED3955D7F
:102F9100401DE55EC3955D855FF0A4FFAEF0E56081
:102FA1008E048F05FF120085ED255DF55C801DE522
:102FB1005DC3955E855FF0A4FFAEF0E5608E048F82
:102FC10005FF120085EDF404255DF55C22E55ED375
:102FD100955D401DE55EC3955D855FF0A4FFAEF094
:102FE100E5608E048F05FF120085ED255DF55C809F
:102FF1001DE55DC3955E855FF0A4FFAEF0E5608ED3
:10300100048F05FF120085EDF404255DF55C22E5D2
:103011003775F00484FF7E008F5CE53775F004841A
:10302100ADF07C008D5F756404753201753300E588
:103031005CC3943F5005122F5480069001A4E0F523
:103041005C855C52755100900037E075F020A4FF5B
:10305100AEF09000B6E08E048F05FF1200858D5C06
:1030610090009EE0D3953750030231169000C2E0E4
:10307100D395374010ED9001A5124ABBE0F5547588
:10308100530002311390008DE0D395374043E55C46
:103091009001A5124ABBE0F55DE55C9001C5124ABD
:1030A100BBE0F55E9000C2E0F4042537F55F9000C7
:1030B1008DE0FE9000C2E0F4042EF560E55DB55EA2
:1030C10005855D5C8003122FCE855C5475530080AD
:1030D10041E55C9001C5124ABBE0F55DE55C9001FC
:1030E100E5124ABBE0F55E90008DE0F4042537F56A
:1030F1005F90009EE0FE90008DE0F4042EF560E507
:103101005DB55E05855D5C8003122FCE855C5475CF
:1031110053000231BD9000C5E0D395375011E55CF5
:10312100900225124ABBE0F5547553000231BD905F
:10313100008EE0D395375043E55C900205124ABBFF
:10314100E0F55DE55C900225124ABBE0F55E90007A
:103151008EE0F4042537F55F9000C5E0FE90008E07
:10316100E0F4042EF560E55DB55E05855D5C8003E8
:10317100122FCE855C547553008041E55C9001E5CA
:10318100124ABBE0F55DE55C900205124ABBE0F531
:103191005E90009EE0F4042537F55F90008EE0FE1E
:1031A10090009EE0F4042EF560E55DB55E05855D59
:1031B1005C8003122FCE855C54755300229000D69B
:1031C100E0F561756411753202753300AE24AF25E7
:1031D100E56175F00FA4FDACF0EDD39FEC9E4021AD
:1031E100E5618E048F05FF120085ED75F010A4FFD7
:1031F100AEF0E53775F01184FD7C00ED2FF56280AE
:103201000EE53775F01184FF7E00EF24F0F562853D
:10321100625CE53775F01184AFF07E008F5F122F8D
:1032210054855C63AE24AF259000D6E075F00FA401
:10323100FDACF0EDD39FEC9E402875320275331042
:1032410085625C122F5485635D855C5EAE24AF257B
:10325100E5618E048F05FF124A9A8D5F85616012C8
:103261002FCE855C527551007554647553002290C0
:1032710000D6E0F561756411753202753300AE2434
:10328100AF25E56175F00FA4FDACF0EDD39FEC9E89
:103291004021E5618E048F05FF120085ED75F01068
:1032A100A4FFAEF0E53975F01184FD7C00ED2FF53A
:1032B10062800EE53975F01184FF7E00EF24F0F590
:1032C1006285625CE53975F01184AFF07E008F5F35
:1032D100122F54855C63AE24AF259000D6E075F0C3
:1032E1000FA4FDACF0EDD39FEC9E40287532027522
:1032F100331085625C122F5485635D855C5EAE245C
:10330100AF25E5618E048F05FF124A9A8D5F8561B5
:1033110060122FCE855C527551009000A0E0B4047C
:1033210053E53775F00484FF7E008F5CE53775F057
:103331000484ADF07C008D5F7564047532017533D2
:1033410000E55CC3943F5005122F5480069001A400
:10335100E0F55CAE51AF52E55C124A7F74648E04B5
:103361008F05FF120085AE51AF52EF2DFDEE3CFCF3
:103371008C518D527554647553002290006BE0B4EA
:103381000146E53F75F00584FF7E008F5CE53F75E2
:10339100F00584ADF07C008D5F75640575320575AF
:1033A1003300E55CC394175005122F548006900535
:1033B1007CE0F55CAE53AF54E55C2FFF50010E7419
:1033C10064124AD68E538F5490006CE0B40146E5E6
:1033D1004075F00584FF7E008F5CE54075F0058443
:1033E100ADF07C008D5F756405753205753348E578
:1033F1005CC394175005122F5480069005C4E0F564
:103401005CAE53AF54E55C2FFF50010E7464124A59
:10341100D68E538F5490007BE0B40249E542C394A9
:103421004175F00584FF7E008F5CE54275F00584EF
:10343100ADF07C008D5F756405753206753300E56E
:103441005CC394135005122F548006900678E0F562
:103451005CAE53AF54E55C2FFF50010E7464124A09
:10346100D68E538F549000BDE0B402028003023522
:103471001BE53775F01584FF7E008F5CE53775F02D
:103481001584ADF07C008D5F75641575320375335D
:10349100F4E55CC3940B5005122F5480069004642C
:1034A100E0F55CE55C75F0FFA4FFAEF09000BEE0D6
:1034B1008E048F05FF120085ED900060F0E53E75EA
:1034C100F078A4FFAEF074FF8E048F05FF12008523
:1034D1008C328D3374028C068D07124A718F5CAC6D
:1034E10032AD337404FF124A9A8D5F7564047532EC
:1034F1000675336EE55CC3941D5005122F5480068A
:103501009006F0E0F55CAE53AF54E55C2FFF50013F
:103511000E7464124AD68E538F5422900073E0B415
:1035210001179007AAE02554FFAE5350010E9000F9
:10353100C7E0124AD68E538F54900073E0B403163D
:10354100A201B3B3501090005FE0C39405A824B862
:103551000006952540028010900095E02554FFAEAD
:103561005350010E8E538F5490006DE0B4020280CF
:1035710003023749900070E0602FE53FD3941E406D
:1035810028900010E0FEA3E0FF9000ABE075F0038F
:10359100A4FDACF0EFD39DEE9C400E9000CFE0A8CF
:1035A10024B80005D3952550030237499000B8E0AF
:1035B1008537F0A4FFAEF07405124A7F7407124AF2
:1035C100718E328F33900077E0A824B800049525DE
:1035D1005012900078E075F002A4FDACF0EFC39DAD
:1035E100EE9C4003023749E53775F00B84FF7E00FE
:1035F1009005F5124AA6FEE0FFEE90006FE0FEEFA7
:103601008E0088F0A4FFAEF074648E048F05FF1263
:1036110000858C328D33900037E075F018A4FFAE31
:10362100F09000B6E08E048F05FF1200858C068DA8
:103631000790060D124AA6AE32AF33E0124A7F74EC
:10364100648E048F05FF1200858C328D33E53DA811
:1036510032B80077D395334072E53DC39533FFE42B
:103661009532FE8E328F337428BE00039F500C7545
:103671003328753200740D90003AF0AE32AF3390BA
:103681000070E0124A7F74288E048F05FF120085B6
:103691008C328D33AE51AF52740A8E048F05FF12F6
:1036A10000858D068C07AC32AD33CFCECF1200032F
:1036B100740A8E048F05FF1200858C328D33AE5152
:1036C100AF52124ADE8E518F52807DE53DA832B84D
:1036D100000495335072AE32AF33E53D124AD68EB7
:1036E100328F337428BE00039F500C753328753216
:1036F10000740D90003AF0AE32AF33900070E012DA
:103701004A7F74288E048F05FF1200858C328D3319
:10371100AE51AF52740A8E048F05FF1200858D06DB
:103721008C07AC32AD33CFCECF120003740A8E04B6
:103731008F05FF1200858C328D33AE51AF52EF2DC4
:10374100FDEE3CFC8C518D5222AE51AF52AC53ADCB
:103751005412000374648E048F05FF1200858C518E
:103761008D52900068E08C068D07124A7F74648E3A
:10377100048F05FF1200858C518D52A2084017AEAF
:1037810024AF257405BE00039F5002D208E539D34A
:1037910094CC4002D2029000CAE0B402089000CC5E
:1037A100E0640160028017AE51AF52E543124A7FD7
:1037B10074E78E048F05FF1200858C518D529000A5
:1037C1008AE05402601B900081E0A824B80012D363
:1037D1009525400DA208B3B35007E539C3949A402B
:1037E100028028AE5AAF5B90007FE075F002A4FD25
:1037F100ACF0EF2DFDEE3CFC74022DFD50010CE50B
:1038010039BC0007D39D400375680185395B755A42
:1038110000E56870030238A09000DDE0C3956840C0
:1038210070E53F75F00584FF7E00900565124AA69C
:10383100E0F533753200AE32AF3390008FE0124ABB
:103841007F74648E048F05FF1200858C348D359052
:1038510000DDE004C395688C068D07124A7F900055
:10386100DDE08E048F05FF1200858C348D359000CC
:1038710080E08C068D07124A7F740A8E048F05FF43
:10388100120085AE51AF52EF2DFDEE3CFC8C518DF7
:103891005205689000DDE0C395685003756800909B
:1038A100008AE05401601B90007EE0A824B8001259
:1038B100D39525400DA208B3B35007E537C394CC87
:1038C1004002802590007CE075F003A4FFAEF0E596
:1038D100652FFF50010E74032FFF50010EE537BE17
:1038E1000007D39F4003756901853765E56970035A
:1038F10002397B9000DEE0C395694070E53F75F0C9
:103901000584FF7E00900565124AA6E0F533753205
:1039110000AE32AF3390008FE0124A7F74648E04A0
:103921008F05FF1200858C348D359000DEE004C3D5
:1039310095698C068D07124A7F9000DEE08E048F18
:1039410005FF1200858C348D3590007DE08C068D4D
:1039510007124A7F740A8E048F05FF120085AE514B
:10396100AF52EF2DFDEE3CFC8C518D52056990005C
:10397100DEE0C39569500375690090008FE0A8519E
:10398100B800049552500990008FE0F5527551002E
:10399100229000CBE0B401028003023A9DA208B359
:1039A1005003023A9B900096E0B40168AE51AF52C9
:1039B100AC24AD25120003743C8E048F05FF120068
:1039C100859000A6E0BC00109D400D9000A8E0A8E5
:1039D10051B8000495525002D203AE51AF52AC24FB
:1039E100AD25120003743C8E048F05FF12008590F3
:1039F10000A6E0C3940ABC0015D39D40119000A815
:103A0100E0C39405A851B80005D395525002800235
:103A1100C2038068AE51AF52AC24AD2512000374CD
:103A2100788E048F05FF1200859000A6E0BC00107F
:103A31009D400D9000A8E0A851B800049552500493
:103A4100D2038038AE51AF52AC24AD2512000374BD
:103A5100788E048F05FF1200859000A6E0C3940ABA
:103A6100BC0015D39D40119000A8E0C39405A85156
:103A7100B80005D3955250028002C203A203B3409D
:103A810019AE51AF529000A7E0124A7F74648E04C0
:103A91008F05FF1200858C518D528002C203900068
:103AA100CBE0B40258E53775F00884FF7E008F5CE7
:103AB100E53775F00884ADF07C008D5F756408759D
:103AC10032017533E0E55CC3943F5005122F5480F9
:103AD10006900264E0F55CE55C75F05EA4FFAEF073
:103AE100740A8E048F05FF1200858C558D56740261
:103AF100BC000AD39D4006755602755500A200B35D
:103B01004006A202B3B35009900016E4F0A3F0807E
:103B110024AE51AF527400D39F74019E400C9000AB
:103B210016E551F0A3E552F0800B74FF900016F8F2
:103B3100E4F0E8A3F09000ADE0D394024006A208BF
:103B4100B3B34002800DAE51AF527402124A7F8E60
:103B5100518F52900096E0B4010DAE51AF527402F4
:103B6100124A7F8E518F52AE51AF52745E124A7F0C
:103B7100740A8E048F05FF1200858C518D527402D8
:103B8100BC000AD39D400675520275510090001485
:103B9100E551F0A3E552F022900037E09003651261
:103BA1004ABBE0F566756764900037E0FE9000A1BE
:103BB100E0D39E4037E53775F00884FF7E008F5CC7
:103BC100E53775F00884ADF07C008D5F756408758C
:103BD1003203753396E55CC3941F5005122F548050
:103BE1000690041AE0F55C855C678035E53775F071
:103BF1000884FF7E008F5CE53775F00884ADF07CAA
:103C0100008D5F7564087532037533B6E55CC39446
:103C11001F5005122F54800690043AE0F55C855C34
:103C210067229000D7E0F561756411753204753330
:103C310000AE24AF25E56175F00FA4FDACF0EDD326
:103C41009FEC9E4021E5618E048F05FF120085EDFA
:103C510075F010A4FFAEF0E53775F01184FD7C001E
:103C6100ED2FF562800EE53775F01184FF7E00EFD0
:103C710024F0F56285625CE53775F01184AFF07E62
:103C8100008F5F122F54855C63AE24AF259000D75F
:103C9100E075F00FA4FDACF0EDD39FEC9E402875CC
:103CA100320475331085625C122F5485635D855C27
:103CB1005EAE24AF25E5618E048F05FF124A9A8D11
:103CC1005F856160122FCE855C6675676422900006
:103CD100D7E0F561756411753204753300AE24AF18
:103CE10025E56175F00FA4FDACF0EDD39FEC9E408E
:103CF10021E5618E048F05FF120085ED75F010A49A
:103D0100FFAEF0E53975F01184FD7C00ED2FF56211
:103D1100800EE53975F01184FF7E00EF24F0F56225
:103D210085625CE53975F01184AFF07E008F5F121A
:103D31002F54855C63AE24AF259000D7E075F00F5A
:103D4100A4FDACF0EDD39FEC9E4028753204753391
:103D51001085625C122F5485635D855C5EAE24AF75
:103D610025E5618E048F05FF124A9A8D5F8561609A
:103D7100122FCE855C667567649000D2E0B4047939
:103D8100900037E0FE9000A1E0D39E4037E5377503
:103D9100F00884FF7E008F5CE53775F00884ADF094
:103DA1007C008D5F756408753203753396E55CC3DD
:103DB100941F5005122F54800690041AE0F55C857B
:103DC1005C678035E53775F00884FF7E008F5CE520
:103DD1003775F00884ADF07C008D5F75640875322D
:103DE100037533B6E55CC3941F5005122F5480064A
:103DF10090043AE0F55C855C672290006BE0B401C9
:103E01003BE53F75F00584FF7E008F5CE53F75F073
:103E11000584ADF07C008D5F7564057532057533E1
:103E210018E55CC394175005122F54800690059431
:103E3100E0F55CE567255CC39464F56790006CE090
:103E4100B4013BE54075F00584FF7E008F5CE540E1
:103E510075F00584ADF07C008D5F756405753205E4
:103E6100753360E55CC394175005122F548006909A
:103E710005DCE0F55CE567255CC39464F567E56600
:103E81002567F559900073E0B402109007A9E02569
:103E910059FE9000C7E0F4042EF5599000CAE0D312
:103EA10094014040E543C394E7501D74E7C3954333
:103EB100FE9007ABE08E00F5F0E884FF7E008F5C9A
:103EC100E559255CF559801CE543C394E7FE90074D
:103ED100ABE08E00F5F0E884FF7E008F5CE559C30E
:103EE100955CF559A2084006E5662464F559E55943
:103EF100D394644009E559C39464F5598003755915
:103F0100009000A3E0C3955950069000A3E0F55935
:103F110022D2009000B9E0A824B800049525503BB6
:103F21009000B9E0A824B800049525500375590FF5
:103F31009000B9E004A824B80004952550037559F0
:103F41000A9000B9E02402A824B800049525500580
:103F5100755905C200740990003AF07E017F009006
:103F610000A9E0124A7F9000B8E08E048F05FF128D
:103F71000085E537BC000CD39D4008C200740A904F
:103F8100003AF09000AAE0C3953F500D9000BCE0CC
:103F9100A824B80006952540028008C200740B9041
:103FA100003AF0A2004003755905900073E0B40394
:103FB10006A201B3B34002802B90005FE0C39405D9
:103FC100A824B800049525500C900094E0F559748C
:103FD1000C90003AF090005FE0A824B80004952509
:103FE1005002C200855944900065E02559FE9000B9
:103FF10037E075F01E84FC7F00EE2CF5592290000D
:1040010037E075F00584FF7E008F5C900037E07526
:10401100F00584ADF07C008D5F7564057532037524
:1040210033D69000B6E01475F00584FF7E00E55CA0
:10403100BE00039F5005122F54800BE55C90043B9A
:10404100124ABBE0F55CE55C9007ACF09007ACE090
:10405100FE9000A5E0C39E50089000A5E09007AC3B
:10406100F022E53F75F00584FF7E00900565124A58
:10407100A6E0F56BE56BD394644010E56BC39464E3
:1040810075F00F84FF7E008F6B8003756B009000CD
:1040910088E0256BF56B2290079FE0FEA3E0FF749B
:1040A10004124A71E537124A7F740F8E048F05FF9F
:1040B10012008590079DECF0A3EDF090007BE0B439
:1040C1000262E542C3944175F00584FF7E008F5C76
:1040D100E54275F00584ADF07C008D5F7564057572
:1040E1003206753314E55CC394175005122F5480C2
:1040F1000690068CE0F55C90079DE0FEA3E0FF745E
:104101000A8E048F05FF120085E55C8C068D07126F
:104111004A7F740A8E048F05FF12008590079DEC7B
:10412100F0A3EDF090079DE0FEA3E0FF9007A3E070
:10413100FCA3E0FDEDD39FEC9E400F9007A3E0F8B8
:10414100A3E090079DC8F0A3C8F022900082E0B4DC
:10415100010385254F900082E0B402129000B8E07F
:104161008537F0A4FFAEF07408124A718F4F9000AA
:1041710082E0B4030385394F900082E0B4040385E3
:104181003F4F900082E0B40507E540C39414F54F1A
:10419100900082E0B4060385414F900082E0B407AD
:1041A1000385424F900082E0B4080385434F90009D
:1041B10082E0B40903853E4F900083E0FE900084C5
:1041C100E0D39E404B900082E0B40418900084E05C
:1041D100C3954F5002D204900083E0D3954F400223
:1041E100C204802A900083E0C3954F500990008457
:1041F100E0D3954F50028002D204900083E0D39522
:104201004F5009900084E0C3954F5002C204802AA8
:10421100900083E0D3954F4009900084E0C3954F0F
:1042210040028002C204900083E0C3954F40099090
:104231000084E0D3954F4002D20422900085E0B47F
:10424100010385254F900085E0B402129000B8E08B
:104251008537F0A4FFAEF07408124A718F4F9000B9
:1042610085E0B4030385394F900085E0B4040385EC
:104271003F4F900085E0B40507E540C39414F54F26
:10428100900085E0B4060385414F900085E0B407B6
:104291000385424F900085E0B4080385434F9000A9
:1042A10085E0B40903853E4F900086E0FE900087CB
:1042B100E0D39E4040900086E0C3954F50099000A6
:1042C10087E0D3954F50028002D206900086E0D35A
:1042D100954F5009900087E0C3954F5002C2069058
:1042E1000085E0B401099000C4E0D3953950028003
:1042F10002C206802A900086E0D3954F40099000C3
:1043010087E0C3954F40028002C206900086E0C359
:10431100954F4009900087E0D3954F4002D2062285
:10432100AE57AF5874F5D39F74019E400878571269
:104331004AE602441C755801755700AE24AF25E5C5
:104341006BBE000DD39F400990009AE0D3956C405D
:1043510002801B756C00E56BC39525F54F90009DA0
:10436100E0D3956A4006E56A254FF56A8002056C3F
:10437100900076E0D39539401CE537C39538401558
:10438100AE24AF25E56BBE00039F500990009BE072
:10439100D3956D400280579007ADE0A824B8000482
:1043A10095255003756F009007ADE0A824B8000B68
:1043B100D395254006E5259007ADF0E56F702AE518
:1043C10025C3956BF54FE54FD394054003754F0514
:1043D10090009CE0C3956A5007E54FC3956A40027F
:1043E1008007E56AC3954FF56A756D008002056D1A
:1043F100E56F7016900076E0C39539500DE56B249A
:1044010005A824B8000695254002800F900089E098
:10441100F56A756F0174789007ADF022AE57AF5809
:1044210074E9D39F74039E40087857124AE6024507
:10443100CA755801755700756A32A21D402A756AFE
:1044410019900089E075F002A4FFAEF0E56CBE00A2
:1044510006D39F4002D21D056C756F0374789007D7
:10446100ADF0756E000245B9AE24AF25E56B6F4E18
:1044710070030245B9E56BBE000DD39F4009900062
:104481009AE0D3956C40028017756C00A208B3B313
:104491005007E56FC3940340028003756A19800DCC
:1044A100E56BC39525F54FE56C254FF56C900076CE
:1044B100E0D39539400E9007ADE0A824B80007D3AA
:1044C10095254002800C056E900089E0B56E03755C
:1044D1006F00E56FB4030DE56B2402A824B8000654
:1044E10095254002800A056EE56EB43C03756F02A6
:1044F100E56FB402299007ADE0A824B8000ED3956A
:10450100254009E5259007ADF0756E00900076E035
:10451100C395395009756E0074789007ADF0E56F59
:10452100705A900076E0D39539401CE537D3953821
:104531004015AE24AF25E56BBE00039F50099000E6
:104541009BE0D3956D40028008756D00756A4B80C4
:1045510028E525C3956BF54FE54FD39405400375C9
:104561004F05900076E0D395394008E56D254FF56C
:104571006D8006E56D2406F56D756E00E56F7016AC
:10458100900076E0C39539500DE56B2405A824B859
:104591000006952540028003756F01E56FB401188F
:1045A100756A19056E900089E0B56E06756F027522
:1045B1006E0074789007ADF0E56A75F00AA4FFAE5D
:0A45C100F09007A7EEF0A3EFF02240
:094ABB002582F5825002058322D8
:0F4A620025E050020583258250020583F582224C
:10006400EF2F500205832582F582E5833E2EF5832A
:010074002269
:104AD600CFC39FFF50011E22C3EF9DFFEE9CFE2217
:094AC400E493F608740193F62254
:084AE6000806B60002180622C2
:0D4A8D00A3E004F07006124AB1E004F0222C
:0E003900A3E014F0B4FF06124AB1E014F02266
:0E4A7100048007C3CE13CECF13CFD5E0F622BC
:10498100BC000FBE0008ED8FF084FFADF022E4FE05
:10499100FF22BE000DEF60FE54F0606F20E70302BE
:1049A1004A37EAC0E0EBC0E078017A0075F001EE29
:1049B10020E710EF25E0FFEE33FE0AC5F023C5F036
:1049C10030E7F0EA5407F9096A7A007B00600108D0
:1049D100C3EC9E40167004ED9F4010ED9FFDEC9ED0
:1049E100FCE5F0CA4ACA03F5F08005E5F003F5F0ED
:1049F100C3EE13FEEF13FFD9D77908CACBCAD8D0BB
:104A0100EAFEEBFFD0E0FBD0E0FA22EC8FF084FC71
:104A1100ED54F045F0C48FF084FEEDC454F045F040
:104A2100C48FF084FDEEC4FE54F02DFFEE540F3C14
:104A3100FEADF07C0022790078008FF0EC7E08203A
:104A4100E70DC3CD33CD33C933C9C833C8DEF084D4
:104A510049F9E5F08FF0BE00E6FD7C00E9FFE8FED4
:014A61002232
:0E4A7F00F88FF0A4FFE5F0CE88F0A42EFE2202
:10000300EF8DF0A4F9A8F0EF8CF0A428F8EE8DF0B2
:06001300A428FEE9FF2213
:10007500600D782B02007F007830D8FED5E0F8229D
:10008500EEC0E07E00124981EFFDEEFCD0E0FE22DD
:0C4A9A00EEC0E07E00124981D0E0FE2258
:03001B0002001EC2
:03009B0002004917
:03000000024ACDE4
:094ACD0075817075D0000204B27D
:104AA600E5822FF582E5833EF583220582D58202D3
:054AB6001583158222AA
:10001E00C0E0C0F0C083C082C0D075D00012045DB5
:0B002E00D0D0D082D083D0F0D0E032E0
:10004900C0E0C0F0C083C082C0D075D00012046087
:0B005900D0D0D082D083D0F0D0E032B5
:00000001FF
